:020000040800F2
:10000000D006002059010008A10400089D04000842
:1000100000000000000000000000000000000000E0
:10002000000000000000000000000000A107000820
:10003000000000000000000015050008870100080E
:1000400089010008000000008901000889010008FA
:100050008901000889010008890100088901000858
:1000600000000000890100088901000889010008DA
:1000700089010008890100088901000800000000CA
:10008000890100080000000000000000890100084C
:100090008901000889010008890100088901000818
:1000A00089010008890100088901000891090008F8
:1000B0008901000800F002F800F03EF80CA030C8FA
:1000C000083824182D18A246671EAB4654465D46D4
:1000D000AC4201D100F030F87E460F3E0FCCB64660
:1000E0000126334200D0FB1AA246AB4633431847E1
:1000F000B40C0000D40C0000103A02D378C878C1C8
:10010000FAD8520701D330C830C101D504680C6059
:10011000704700000023002400250026103A01D378
:1001200078C1FBD8520700D330C100D50B607047AF
:100130001FB51FBD10B510BD00F0FAF81146FFF74E
:10014000F7FF00F0A9FD00F012F903B4FFF7F2FF8A
:1001500003BC00F05AFD00000F4880F308880F48E8
:100160000168090E0E4A914205D10E480E49016000
:100170000E480F4901600F4880470F480047FEE7CF
:10018000FEE7FEE7FEE7FEE7FEE700000B480C494E
:100190000C4A0D4B70470000D00600200400000000
:1001A0001F00000018100240010000000000014084
:1001B0000000000015090008B5000008D00000206C
:1001C000D0060020D0020020D0020020704700227C
:1001D00003098B422CD3030A8B4211D300239C4684
:1001E0004EE003460B433CD4002243088B4231D3FC
:1001F00003098B421CD3030A8B4201D394463FE090
:10020000C3098B4201D3CB01C01A524183098B42EF
:1002100001D38B01C01A524143098B4201D34B01D8
:10022000C01A524103098B4201D30B01C01A52413B
:10023000C3088B4201D3CB00C01A524183088B42C2
:1002400001D38B00C01A524143088B4201D34B00AB
:10025000C01A5241411A00D201465241104670471D
:100260005DE0CA0F00D04942031000D34042534022
:1002700000229C4603098B422DD3030A8B4212D3E2
:10028000FC22890112BA030A8B420CD38901921114
:100290008B4208D3890192118B4204D389013AD051
:1002A000921100E08909C3098B4201D3CB01C01A26
:1002B000524183098B4201D38B01C01A5241430939
:1002C0008B4201D34B01C01A524103098B4201D327
:1002D0000B01C01A5241C3088B4201D3CB00C01A94
:1002E000524183088B4201D38B00C01A5241D9D2AC
:1002F00043088B4201D34B00C01A5241411A00D22D
:100300000146634652415B10104601D34042002B28
:1003100000D54942704763465B1000D3404201B5A7
:100320000020C046C04602BD704770477047704706
:10033000754600F025F8AE46050069465346C008EC
:10034000C000854618B020B5FFF720FF60BC00272D
:100350004908B6460026C0C5C0C5C0C5C0C5C0C591
:10036000C0C5C0C5C0C5403D49008D46704710B5E9
:100370000446C046C0462046FFF7E7FE10BD000019
:100380000048704770000020F0B50A4600210023A5
:10039000002400BF3DE001258D402B4615681D401F
:1003A0002C469C4234D11579012D02D01579022DAD
:1003B00016D185684F000326BE40B5438560557948
:1003C0004E00B540866835438560858801268E409D
:1003D000B5438580858896798E40B6B23543858051
:1003E00005684F000326BE40B543056015794E00F1
:1003F000B540066835430560C5684F000326BE401A
:10040000B543C560D5794E00B540C6683543C56073
:10041000491C1029BFD3F0BDF0B5002300244D07BF
:10042000EE0E1546B5402B46CD10AE0005462035E4
:10043000AD594E07F70E0F26BE40B543CE10B6009D
:1004400007462037BD51CD10AE003D46AD591D4386
:100450002C46CD10AD003E467451F0BD018570476D
:100460001CB50121C80400F057F8032000020090D9
:100470000021684641710121017100218171012132
:10048000C17169460448FFF77FFF03210902024852
:10049000FFF7E4FF1CBD00000008004800BFFEE7B6
:1004A0007047000000218278002A27D0184A0323D1
:1004B0001B02D21803789B109B00D1580278920738
:1004C000D30EFF229A400B46934319464278920777
:1004D000120E03789B07DB0E9A4011430C4A03234C
:1004E0001B02D21803789B109B00D1500278D306D0
:1004F000DB0E01229A40064B1A6007E00278D30611
:10050000DB0E01229A40024B80331A6070470000D4
:1005100000E100E070470000002905D0054A52695B
:100520000243044B5A6104E0024A52698243014B80
:100530005A61704700100240002905D0054A9269AF
:100540000243044B9A6104E0024A92698243014BE0
:100550009A61704700100240FEB50446002500264F
:1005600000200290019000900027864840680C21EE
:1005700008400546002D06D0042D07D0082D08D0D0
:100580000C2D2CD128E0804820602BE07E48206094
:1005900028E07C4840680F218904084006467948D5
:1005A00040680321C90308400290B00C861C0298E1
:1005B000002803D17548374647430BE07148C06AAD
:1005C0000007000F401C01906F480199FFF7FFFDE5
:1005D00070430746276005E06D48206002E06A48E6
:1005E000206000BF00BF67484068F0210840054612
:1005F0002D096848405D009020680099C8406060FF
:100600006048406807210902084005462D0A6148F4
:10061000405D009061680098C140A1605948006B3E
:10062000FF2101310840884202D05B48E0600DE0C4
:1006300054484068012189030840884203D0A068DB
:100640004008E06002E0A0688008E0604D48006B70
:1006500040210840402802D05048206102E001209B
:10066000C00320614748006B10210840102802D0C9
:100670004548606101E0206860614248006B800786
:10068000800F002802D1A068A06119E03D48006BEE
:100690008007800F012802D12068A06110E039484E
:1006A000006B8007800F022802D18003A06107E061
:1006B0003448006B8007800F032801D13248A061C5
:1006C0003048006B032109040840002802D1A068CB
:1006D000E06120E02B48006B032109040840012160
:1006E0000904884202D12068E06114E02548006BCB
:1006F00003210904084001214904884202D18010E5
:10070000E06108E01F48006B0321090408408842AB
:1007100001D11D48E0611B48006B0321890408409A
:10072000002802D1A068206220E01648006B032157
:100730008904084001218904884202D1206820628E
:1007400014E01048006B0321890408400121C9040A
:10075000884202D10011206208E00A48006B0321A0
:1007600089040840884201D1074820620548006B8F
:1007700080210840802802D00548606200E067625E
:10078000FEBD00000010024000127A0000093D008A
:10079000006CDC0214000020809FD5001280000055
:1007A000704700000CB50020019000904E48006892
:1007B0000121090408434C49086000BF4A48006809
:1007C00001214904084000900198401C01900098C4
:1007D000002804D10521090301988842EED142483E
:1007E0000068012149040840002802D0012000903F
:1007F00001E000200090009801283AD111203B49E7
:100800000860394840683849486008464068486090
:10081000084640687F21C903884333494860084639
:1008200040681121090408432F49486008460068C0
:100830000121090608432C49086000BF2A480068C6
:100840000121490608400028F8D027484068800860
:100850008000254948600846406802210843224933
:10086000486000BF204840680C2108400828F9D1A2
:1008700039E011201D4908601B4840681A4948604A
:10088000084640684860084640687B21C9038843A1
:1008900015494860084640680521C90408431249C3
:1008A0004860084600680121090608430E490860AF
:1008B00000BF0D4800680121490608400028F8D013
:1008C0000948406880088000074948600846406839
:1008D000022108430449486000BF034840680C21D6
:1008E00008400828F9D10CBD001002400020024049
:1008F000042806D10649096904221143044A1161FA
:1009000005E00349096904229143014A11617047D6
:1009100000E000E010B51B480068012108431949B8
:10092000086008464068184908401649486008466B
:10093000006816490840134908600846006801210C
:10094000890488430F490860084640683F2109042C
:1009500088430C4948600846C06A00090001C86223
:100960000846006BFF215431884306490863084656
:10097000406B40084000486300208860FFF712FF8A
:1009800010BD0000001002400CB8FF08FFFFF6FE8B
:1009900010B52D492D4800F06FF8002853D02B4892
:1009A00000F02EF9C4B22A4800880121C90308408A
:1009B000002848D12648008849100840002827D040
:1009C0000A2C1DD00D20224909888904890C214A4E
:1009D00050541F480088401C1D4908800846008864
:1009E0008004800C11460C5419480088401C18499A
:1009F000088008460088184908401549088022E008
:100A0000134800880121C9030843114908801AE0EE
:100A10000D2C07D10E4800880121890308430C4999
:100A2000088010E00A4800888004800C09490C54B2
:100A300007480088401C06490880084600883F286F
:100A400001DD0020088010BD0501050000380140CF
:100A50002C00002030000020FFBF00000162704722
:100A6000002904D0026801231A43026003E00268EF
:100A7000520852000260704770B502460B460024CF
:100A80000021002500201E04350ED9B201268E401B
:100A90003146012D02D11668314006E0022D02D107
:100AA0005668314001E0966831401C0C0126A64092
:100AB0003446D6693440002903D0002C01D00120EF
:100AC00000E0002070BDF8B5034600240026009623
:100AD0000025002018460E04340ECEB200960127E1
:100AE000009EB7403D46022C01D1001D02E0032CC0
:100AF00000D10830002A03D006682E43066002E0C9
:100B00000668AE430660F8BDF0B58BB004460D46EE
:100B1000002700200A90002620684008400020603E
:100B2000666803210903304688430646A8680643E1
:100B3000666026682D480640E968686808432969A8
:100B4000084306432660A66803210902304688430D
:100B5000064668690643A6606846FFF7FDFC244820
:100B6000844202D106980A900DE02248844202D1C4
:100B700007980A9007E02048844202D108980A901A
:100B800001E002980A9020680121C903084000286A
:100B90000CD029680A9A5000FFF719FB074629680C
:100BA0000A9A5000FFF713FB0E4609E029680A98DD
:100BB000FFF70DFB074629680A98FFF708FB0E466A
:100BC00028684008B04200D87F1C20680121C90372
:100BD0000840002806D03807460F38460749084025
:100BE00030430746A7810BB0F0BD0000F3E9FFFFDB
:100BF000003801400044004000480040F0FF000081
:100C00000146888CC005C00D7047014600BF704783
:100C100010B50420C043FFF76BFE07490748006882
:100C2000FFF7D5FA06490870084600787D21C9000B
:100C300048430449088010BD00127A0000000020DB
:100C400024000020260000200146114A12884A4351
:100C5000104B5A6100229A611A46126901231A4305
:100C60000C4B1A6100BF0B4A1069C207D20F002A51
:100C700004D0012212040240002AF4D0054A12696D
:100C800052085200034B1A6100229A61704700001B
:100C90002600002000E000E00024FFF7B9FFE1207B
:100CA000400200F02FF8FFF7DBFB27E0601CC4B226
:100CB0000A20FFF7C9FF322C20DD00241049898A61
:100CC000C905C90F0122514009021202114008460C
:100CD0000B49898A91430143094A91821146898AC5
:100CE0008905C90F012251404902520211400846AC
:100CF0000349898A91430143014A9182D6E7000062
:100D00000008004810B58AB0044601214804FFF7E6
:100D100003FC01218803FFF70FFC01220921C8060B
:100D2000FFF77AFB01220A210920C006FFF774FBB6
:100D3000032040020890032108A84171022101719B
:100D4000002181710121C17108A90920C006FFF7A6
:100D50001BFB0294002003900490059007900C2048
:100D6000069002A90D48FFF7CFFE01210B48FFF7BF
:100D700077FE40210948FFF771FE01220849074824
:100D8000FFF7A1FE1B21684601710321417101217A
:100D9000817101A8FFF786FB0AB010BD0038014041
:100DA00005010500C40D000800000020300000000F
:100DB000F8000008F40D000830000020A006000034
:100DC00014010008006CDC020000000000000000BC
:100DD00001020304060708090000000001020304E1
:100DE00001020304060708090000000000000000DB
:040DF00000000000FF
:04000005080000B53A
:00000001FF
